:1000000010C017C016C015C014C013C012C011C054
:1000100010C00FC00EC00DC00CC00BC00AC009C07C
:1000200008C011241FBECFE5D1E0DEBFCDBF02D096
:1000300094C0E6CF80E886BD16BCC19AB99AC09A32
:10004000B89AC29ABA9A80E0C198982F2AE12A9564
:10005000F1F700C09F5F9F3FC9F7C19A90E021E090
:10006000290F981731F09AE19A95F1F700C0922F75
:10007000F6CF822F2F3F41F780E0C19AC098982F8A
:100080002AE12A95F1F700C09F5F9F3FC9F7C19809
:10009000C09A90E021E0290F981731F09AE19A95E3
:1000A000F1F700C0922FF6CF822F2F3F31F780E07B
:1000B000C09AC298982F2AE12A95F1F700C09F5F55
:1000C0009F3FC9F7C098C29A90E021E0290F981786
:1000D00031F09AE19A95F1F700C0922FF6CF822F76
:1000E0002F3F31F780E0C29AC098C198982F2AE13B
:1000F0002A95F1F700C09F5F9F3FC9F7C29AC09A47
:10010000C19A90E021E0290F981731F09AE19A9571
:10011000F1F700C0922FF6CF822F2F3F21F780E01A
:10012000C29AC09AC19A982F2AE12A95F1F700C085
:100130009F5F9F3FC9F7C298C098C19890E021E0A7
:10014000290F981731F09AE19A95F1F700C0922F94
:0E015000F6CF822F2F3F21F776CFF894FFCF06
:00000001FF
